:020000040800F2
:1000000000060020A1020008FD0F00087D0F000877
:10001000D50F00087D0F0008A90F0008A3020008F3
:10002000A3020008A3020008A3020008512300084D
:10003000A3020008A3020008A3020008A30200080C
:10004000A3020008A3020008A3020008A3020008FC
:10005000A3020008A3020008D937000805380008E9
:10006000313800085D38000889380008A30200080C
:10007000A3020008A3020008A3020008A3020008CC
:10008000A3020008A3020008A3020008A3020008BC
:10009000A3020008A3020008A3020008B538000864
:1000A000A3020008A3020008A3020008A30200089C
:1000B000A3020008A3020008A3020008A30200088C
:1000C000A3020008A3020008A3020008A30200087C
:1000D000A3020008A3020008A3020008A30200086C
:1000E00019390008A3020008A3020008A3020008AF
:1000F000A3020008A3020008A3020008A30200084C
:10010000A3020008A30200088D390008A30200081A
:10011000A3020008A3020008A3020008A30200082B
:10012000A3020008A3020008A3020008A30200081B
:10013000A3020008A3020008A3020008A30200080B
:10014000A3020008A3020008A3020008A3020008FB
:10015000A3020008A3020008A3020008A3020008EB
:10016000A3020008A3020008A3020008A3020008DB
:10017000A3020008BD2E0008A3020008A302000885
:10018000A3020008A3020008A3020008A3020008BB
:10019000A3020008A3020008A3020008A3020008AB
:1001A000A3020008A3020008A3020008A30200089B
:1001B000A3020008A3020008A3020008A30200088B
:1001C000A3020008A3020008A3020008A30200087B
:1001D000A3020008A92E0008A3020008A302000839
:1001E000A3020008A3020008A3020008A30200085B
:1001F000A3020008A3020008A3020008A30200084B
:10020000A3020008A3020008A3020008A30200083A
:10021000A3020008A3020008A3020008A30200082A
:10022000A3020008A3020008A3020008A30200081A
:10023000A3020008A3020008A3020008A30200080A
:10024000A3020008A3020008A3020008A3020008FA
:10025000A3020008A3020008A3020008A3020008EA
:10026000A3020008A3020008A3020008A3020008DA
:10027000A3020008A3020008A3020008A3020008CA
:10028000A3020008A3020008A3020008A3020008BA
:10029000A3020008A3020008A3020008A3020008AA
:1002A00002E000F000F8FEE772B63A4880F30888F2
:1002B000394880F3098839484EF60851CEF20001DA
:1002C000086040F20000CCF200004EF63471CEF22D
:1002D00000010860BFF34F8FBFF36F8F40F2000043
:1002E000C0F2F0004EF68851CEF200010860BFF374
:1002F0004F8FBFF36F8F4FF00000E1EE100A4EF604
:100300003C71CEF200010860062080F31488BFF330
:100310006F8F02F0DBF802F07DF803F017F84FF072
:1003200055301F491B4A91423CBF41F8040BFAE784
:100330001C49194A91423CBF41F8040BFAE71A499B
:100340001A4A1B4B9A423EBF51F8040B42F8040B69
:10035000F8E700201749184A91423CBF41F8040BC6
:10036000FAE702F095F803F075F8144C144DAC421E
:1003700003DA54F8041B8847F9E700F041F8114C00
:10038000114DAC4203DA54F8041B8847F9E702F038
:100390007DB80000000600200022002000000008B8
:1003A0000000002000060020583D00080022002028
:1003B0005C220020602200207C420020A002000875
:1003C000A0020008A0020008A00200082DE9F04FDA
:1003D0002DED108AC1F80CD0D0F80CD0BDEC108AED
:1003E000BDE8F08F002383F311882846A047002042
:1003F00001F090FBFEE701F00BFB00DFFEE70000E1
:1004000038B501F08DFF30B1164B00220A211A7267
:100410005A729972DA7201F059FF054601F08EFFA7
:100420000446D0B9104B9D4219D001339D4241F290
:10043000883512BF044600250124002001F050FF3A
:100440000CB100F079F800F06DFD00F015FC2846C5
:1004500000F020F900F070F8F9E70025EDE7054617
:10046000EBE700BF00220020010007B008B500F054
:10047000D5FBA0F120035842584108BD07B541F211
:100480001203022101A8ADF8043000F0E5FB03B02F
:100490005DF804FB38B5202383F311881748C3683F
:1004A0000BB101F0BDFB0023154A4FF47A711348DC
:1004B00001F07AFB002383F31188124C236813B1F7
:1004C0002368013B2360636813B16368013B636089
:1004D0000D4D2B7833B963687BB9022000F09CFC8A
:1004E000322363602B78032B07D163682BB902207A
:1004F00000F092FC4FF47A73636038BD60220020F4
:10050000950400087C23002074220020084B1870FA
:1005100003280CD8DFE800F008050208022000F0EC
:1005200071BC022000F064BC024B00225A6070478C
:10053000742200207C230020F8B5504B504A1C4602
:100540001968013100F0998004339342F8D1626850
:100550004C4B9A4240F291804B4B9B6803F10063F5
:1005600003F5C0239A4280F08880002000F09EFBB3
:100570000220FFF7CBFF454B0021D3F8E820C3F85A
:10058000E810D3F81021C3F81011D3F81021D3F8D4
:10059000EC20C3F8EC10D3F81421C3F81411D3F8ED
:1005A0001421D3F8F020C3F8F010D3F81821C3F8C1
:1005B0001811D3F81821D3F8802042F00062C3F854
:1005C0008020D3F8802022F00062C3F88020D3F886
:1005D0008020D3F8802042F00072C3F88020D3F846
:1005E000802022F00072C3F88020D3F8803072B6E9
:1005F0004FF0E023C3F8084DD4E90004BFF34F8F58
:10060000BFF36F8F224AC2F88410BFF34F8F536934
:1006100023F480335361BFF34F8FD2F8803043F619
:10062000E076C3F3C905C3F34E335B0103EA060C5E
:1006300029464CEA81770139C2F87472F9D2203B1D
:1006400013F1200FF2D1BFF34F8FBFF36F8FBFF3C2
:100650004F8FBFF36F8F536923F40033536100232F
:10066000C2F85032BFF34F8FBFF36F8F202383F355
:100670001188854680F308882047F8BD00000608E9
:1006800020000608FFFF0508002200200044025851
:1006900000ED00E02DE9F04F93B0B44B2022FF2194
:1006A00000900AA89D6800F0E7FBB14A1378A3B94F
:1006B0000121B0481170C360202383F31188C368FF
:1006C0000BB101F0ADFA0023AB4A4FF47A71A9489F
:1006D00001F06AFA002383F31188009B13B1A74B42
:1006E000009A1A60A64A1378032B03D000231370D4
:1006F000A24A53604FF0000A009CD3465646D146AA
:10070000012000F07FFB24B19C4B1B68002B00F004
:100710002682002000F082FA0390039B002BF2DB7C
:10072000012000F065FB039B213B1F2BE8D801A2B1
:1007300052F823F0B5070008DD070008710800082B
:100740000107000801070008010700080309000865
:10075000D30A0008ED0900084F0A0008770A0008CC
:100760009D0A000801070008AF0A000801070008F9
:10077000210B00085508000801070008650B000858
:10078000C107000855080008010700084F0A0008C3
:100790000107000801070008010700080107000819
:1007A0000107000801070008010700080107000809
:1007B000710800080220FFF759FE002840F0F98177
:1007C000009B022105A8BAF1000F08BF1C4641F2A8
:1007D0001233ADF8143000F03FFA91E74FF47A701D
:1007E00000F01CFA071EEBDB0220FFF73FFE00289B
:1007F000E6D0013F052F00F2DE81DFE807F0030AB3
:100800000D1013360523042105A8059300F024FAE2
:1008100017E004215548F9E704215A48F6E7042176
:100820005948F3E74FF01C08404608F1040800F06F
:100830003FFA0421059005A800F00EFAB8F12C0F3C
:10084000F2D101204FF0000900FA07F747EA0B0B3D
:100850005FFA8BFB00F05CFB26B10BF00B030B2B5C
:1008600008BF0024FFF70AFE4AE704214748CDE706
:10087000002EA5D00BF00B030B2BA1D10220FFF70C
:10088000F5FD074600289BD00120002600F00EFA57
:100890000220FFF73BFE5FFA86F8404600F016FAAA
:1008A0000446B0B1039940460136A1F140025142DD
:1008B000514100F01BFA0028EDD1BA46044641F23E
:1008C0001213022105A83E46ADF8143000F0C4F919
:1008D00016E725460120FFF719FE244B9B68AB4223
:1008E00007D9284600F0E4F9013040F0678104356B
:1008F000F3E70025224BBA463E461D701F4B5D6054
:10090000A8E7002E3FF45CAF0BF00B030B2B7FF43A
:1009100057AF0220FFF7FAFD322000F07FF9B0F167
:100920000008FFF64DAF18F003077FF449AF0F4AF8
:1009300008EB0503926893423FF642AFB8F5807F1B
:100940003FF73EAF124BB845019323DD4FF47A7069
:1009500000F064F90390039A002AFFF631AF039A7E
:100960000137019B03F8012BEDE700BF00220020B7
:100970007823002060220020950400087C230020BA
:100980007422002004220020082200200C220020D3
:1009900078220020C820FFF769FD074600283FF4B1
:1009A0000FAF1F2D11D8C5F120020AAB25F00300AF
:1009B00084494245184428BF4246019200F036FA65
:1009C000019AFF217F4800F057FA4FEAA803C8F3C5
:1009D00087027C492846019300F056FA0646002813
:1009E0003FF46DAF019B05EB830533E70220FFF772
:1009F0003DFD00283FF4E4AE00F096F900283FF4F6
:100A0000DFAE0027B846704B9B68BB4218D91F2F3A
:100A100011D80A9B01330ED027F0030312AA134406
:100A200053F8203C05934046042205A9043700F002
:100A3000E7FA8046E7E7384600F03AF90590F2E732
:100A4000CDF81480042105A800F006F902E7002380
:100A5000642104A8049300F0F5F800287FF4B0AEF8
:100A60000220FFF703FD00283FF4AAAE049800F02F
:100A700051F90590E6E70023642104A8049300F0EF
:100A8000E1F800287FF49CAE0220FFF7EFFC00287D
:100A90003FF496AE049800F03FF9EAE70220FFF732
:100AA000E5FC00283FF48CAE00F04EF9E1E70220AF
:100AB000FFF7DCFC00283FF483AE05A9142000F00A
:100AC00049F907460421049004A800F0C5F8394606
:100AD000B9E7322000F0A2F8071EFFF671AEBB079F
:100AE0007FF46EAE384A07EB0903926893423FF6F3
:100AF00067AE0220FFF7BAFC00283FF461AE27F092
:100B000003074F44B9453FF4A5AE484609F104092F
:100B100000F0CEF80421059005A800F09DF8F1E75B
:100B20004FF47A70FFF7A2FC00283FF449AE00F0C2
:100B3000FBF8002844D00A9B01330BD008220AA9F5
:100B4000002000F0A1F900283AD02022FF210AA8B5
:100B500000F092F9FFF792FC1C4800F0E1FF13B09F
:100B6000BDE8F08F002E3FF42BAE0BF00B030B2BE8
:100B70007FF426AE0023642105A8059300F062F8F7
:100B8000074600287FF41CAE0220FFF76FFC80466A
:100B900000283FF415AEFFF771FC41F2883000F0F9
:100BA000BFFF059800F0E8F946463C4600F0B0F972
:100BB000A6E506464EE64FF0000901E6BA467EE697
:100BC00037467CE67822002000220020A086010023
:100BD0000F4B70B51B780C460133DBB2012B11D8DB
:100BE0000C4D4FF47A732968A2FB033222460E6A39
:100BF00001462846B047844204D1074B0022012019
:100C00001A7070BD4FF4FA7000F08AFF0020F8E708
:100C10001022002070250020B0230020002307B5FB
:100C2000024601210DF107008DF80730FFF7D0FFD4
:100C300020B19DF8070003B05DF804FB4FF0FF30D2
:100C4000F9E700000A46042108B5FFF7C1FF80F06C
:100C50000100C0B2404208BD30B4054C0A4601460E
:100C600023682046DD69034BAC4630BC604700BFBB
:100C700070250020A086010070B50A4E00240A4DA0
:100C800001F0FCF9308028683388834208D901F0EC
:100C9000F1F92B6804440133B4F5C02F2B60F2D373
:100CA00070BD00BFB22300208423002001F0C4BA2D
:100CB00000F1006000F5C0200068704700F100609E
:100CC000920000F5C02001F03BBA0000054B1A6805
:100CD000054B1B889B1A834202D9104401F0CAB904
:100CE0000020704784230020B223002038B504463A
:100CF000074D29B128682044BDE8384001F0D2B939
:100D00002868204401F0BCF90028F3D038BD00BFAA
:100D1000842300200020704700F1FF5000F58F1061
:100D2000D0F8000870470000064991F8243033B12C
:100D300000230822086A81F82430FFF7BFBF012092
:100D4000704700BF88230020014B1868704700BF20
:100D50000010005C244BF0B51A680446234BC2F324
:100D60000B06120C1F885868BE4293F9085028D011
:100D70009F89BE4206D101200C2505FB003358682F
:100D800093F9085041F201039A421CD041F2030347
:100D90009A421AD042F201039A4218D042F2030357
:100DA0009A4208BF5625621E0B46441E0A449342CF
:100DB0000FD214F9016F581C6EB1034600F8016C94
:100DC000F5E70020D8E75A25EDE75925EBE7582548
:100DD000E9E7184605E02C2482421C7001D9981CD2
:100DE0005D70401AF0BD00BF0010005C14220020AE
:100DF000022803D1024B4FF080729A61704700BF06
:100E000000000258022803D1024B4FF480729A610D
:100E1000704700BF00000258022804D1024A5369FB
:100E200083F480735361704700000258002310B5AB
:100E3000934203D0CC5CC4540133F9E710BD0000E9
:100E4000013810B510F9013F3BB191F900409C42C7
:100E500003D11AB10131013AF4E71AB191F9002036
:100E6000981A10BD1046FCE703460246D01A12F944
:100E7000011B0029FAD1704702440346934202D075
:100E800003F8011BFAE770472DE9F8431F4D14469C
:100E90000746884695F8242052BBDFF870909CB333
:100EA00095F824302BB92022FF2148462F62FFF706
:100EB000E3FF95F824004146C0F1080205EB8000ED
:100EC000A24228BF2246D6B29200FFF7AFFF95F8A4
:100ED0002430A41B17441E449044E4B2F6B2082EFA
:100EE00085F82460DBD1FFF71FFF0028D7D108E089
:100EF0002B6A03EB82038342CFD0FFF715FF002854
:100F0000CBD10020BDE8F8830120FBE78823002037
:100F1000024B1A78024B1A70704700BFB0230020B2
:100F20001022002010B5104C104800F0FBF82146AC
:100F30000E4800F023F924680D48D4F89020D2F828
:100F4000043843F00203C2F8043800F0E9FD09490F
:100F5000204600F021FAD4F89020D2F8043823F08B
:100F60000203C2F8043810BD383B00087025002089
:100F700040420F00403B00087047000000B59BB0A6
:100F8000EFF3098168226846FFF750FFEFF305830E
:100F9000044B9A6BDA6A9A6A9A6A9A6A9A6A9A6AA5
:100FA0009B6AFEE700ED00E000B59BB0EFF309811E
:100FB00068226846FFF73AFFEFF30583044B9A6B0C
:100FC0009A6A9A6A9A6A9A6A9A6A9B6AFEE700BF64
:100FD00000ED00E000B59BB0EFF3098168226846A0
:100FE000FFF724FFEFF30583034B5A6B9A6A9A6A63
:100FF0009A6A9A6A9B6AFEE700ED00E0FEE700004D
:1010000030B50A44084D91420DD011F8013B5840CB
:10101000082340F30004013B2C4013F0FF0384EA53
:101020005000F6D1EFE730BD2083B8ED0268436889
:101030001143016003B118477047000013B5406BBE
:1010400000F58054D4F8A4381A681178042914D112
:10105000017C022911D11979012312898B40134295
:101060000BD101A94C3002F071F8D4F8A448024623
:10107000019B2179206800F0DFF902B010BD00006B
:10108000143001F0F3BF00004FF0FF33143001F0D3
:10109000EDBF00004C3002F0C5B800004FF0FF3348
:1010A0004C3002F0BFB80000143001F0C1BF0000A6
:1010B0004FF0FF31143001F0BBBF00004C3002F0A4
:1010C00091B800004FF0FF324C3002F08BB80000B6
:1010D0000020704710B500F58054D4F8A4381A6881
:1010E0001178042917D1017C022914D159790123DF
:1010F00052898B4013420ED1143001F053FF024647
:1011000048B1D4F8A4484FF4407361792068BDE831
:10111000104000F07FB910BD406BFFF7DBBF00004F
:10112000704700007FB5124B01250426044603607A
:101130000023057400F1840243602946C0E90233AC
:101140000C4B0290143001934FF44073009601F061
:1011500005FF094B04F69442294604F14C00029421
:10116000CDE900634FF4407301F0CCFF04B070BDD3
:10117000743A0008191100083D1000080A6820237D
:1011800083F311880B790B3342F823004B79133327
:1011900042F823008B7913B10B3342F8230000F59A
:1011A0008053C3F8A41802230374002383F3118827
:1011B0007047000038B5037F044613B190F85430EF
:1011C000ABB90125201D0221FFF730FF04F1140007
:1011D0006FF00101257700F0CBFC04F14C0084F89E
:1011E00054506FF00101BDE8384000F0C1BC38BD7B
:1011F00010B5012104460430FFF718FF00232377C0
:1012000084F8543010BD000038B504460025143071
:1012100001F0BCFE04F14C00257701F08BFF201D8E
:1012200084F854500121FFF701FF2046BDE8384003
:10123000FFF750BF90F8803003F06003202B06D1F9
:1012400090F881200023212A03D81F2A06D80020E5
:101250007047222AFBD1C0E91D3303E0034A4267ED
:1012600007228267C3670120704700BF2C2200203D
:1012700037B500F58055D5F8A4381A6811780429D7
:101280001AD1017C022917D11979012312898B40C7
:10129000134211D100F14C04204602F00BF858B172
:1012A00001A9204601F052FFD5F8A4480246019B4F
:1012B0002179206800F0C0F803B030BD01F10B03C4
:1012C000F0B550F8236085B004460D46FEB12023EA
:1012D00083F3118804EB8507301D0821FFF7A6FE74
:1012E000FB6806F14C005B691B681BB1019001F0C3
:1012F0003BFF019803A901F029FF024648B1039B77
:101300002946204600F098F8002383F3118805B0A1
:10131000F0BDFB685A691268002AF5D01B8A013BB0
:101320001340F1D104F18002EAE70000133138B52F
:1013300050F82140ECB1202383F3118804F5805349
:10134000D3F8A4281368527903EB8203DB689B6906
:101350005D6845B104216018FFF768FE294604F175
:10136000140001F029FE2046FFF7B4FE002383F3AA
:10137000118838BD7047000001F01CB901234022DC
:10138000002110B5044600F8303BFFF775FD00233F
:10139000C4E9013310BD000010B52023044683F3D7
:1013A00011882422416000210C30FFF765FD2046A2
:1013B00001F022F902232370002383F3118810BD6A
:1013C00070B500EB8103054650690E461446DA609D
:1013D00018B110220021FFF74FFDA06918B11022AB
:1013E0000021FFF749FD31462846BDE8704001F075
:1013F00015BA000083682022002103F0011310B504
:10140000044683601030FFF737FD2046BDE81040EA
:1014100001F090BAF0B4012500EB810447898D40BA
:10142000E4683D43A469458123600023A2606360B2
:10143000F0BC01F0ADBA0000F0B4012500EB81046E
:1014400007898D40E4683D4364690581236000237A
:10145000A2606360F0BC01F023BB000070B5022302
:1014600000250446242203702946C0F888500C3019
:1014700040F8045CFFF700FD204684F8705001F04E
:1014800061F963681B6823B129462046BDE87040B6
:10149000184770BD037880F88C30052303704368CB
:1014A0001B6810B504460BB1042198470023A360C4
:1014B00010BD000090F88C20436802701B680BB1CF
:1014C000052118477047000070B590F87030044649
:1014D00013B1002380F8703004F18002204601F03F
:1014E0004DFA63689B68B3B994F8803013F06005D7
:1014F00035D00021204601F0F7FC0021204601F004
:10150000E7FC63681B6813B1062120469847062351
:1015100084F8703070BD204698470028E4D0B4F8B5
:101520008630A26F9A4288BFA36794F98030A56F76
:10153000002B4FF0200380F20381002D00F0F28099
:10154000092284F8702083F3118800212046D4E911
:101550001D23FFF771FF002383F31188DAE794F866
:10156000812003F07F0343EA022340F202329342D8
:1015700000F0C58021D8B3F5807F48D00DD8012B6D
:101580003FD0022B00F09380002BB2D104F18802EF
:1015900062670222A267E367C1E7B3F5817F00F0CB
:1015A0009B80B3F5407FA4D194F88230012BA0D169
:1015B000B4F8883043F0020332E0B3F5006F4DD049
:1015C00017D8B3F5A06F31D0A3F5C063012B90D825
:1015D0006368204694F882205E6894F88310B4F81B
:1015E0008430B047002884D0436863670368A367EA
:1015F0001AE0B3F5106F36D040F6024293427FF402
:1016000078AF5C4B63670223A3670023C3E794F8BA
:101610008230012B7FF46DAFB4F8883023F00203E1
:10162000A4F88830C4E91D55E56778E7B4F8803040
:10163000B3F5A06F0ED194F88230204684F88A303A
:1016400001F0DEF863681B6813B10121204698475A
:10165000032323700023C4E91D339CE704F18B03AB
:1016600063670123C3E72378042B10D1202383F37E
:1016700011882046FFF7BEFE85F3118803216368B9
:1016800084F88B5021701B680BB12046984794F862
:101690008230002BDED084F88B3004232370636803
:1016A0001B68002BD6D0022120469847D2E794F839
:1016B000843020461D0603F00F010AD501F050F9D1
:1016C000012804D002287FF414AF2B4B9AE72B4B50
:1016D00098E701F037F9F3E794F88230002B7FF4B4
:1016E00008AF94F8843013F00F01B3D01A062046E7
:1016F00002D501F011FCADE701F002FCAAE794F875
:101700008230002B7FF4F5AE94F8843013F00F0193
:10171000A0D01B06204602D501F0E6FB9AE701F0B7
:10172000D7FB97E7142284F8702083F311882B46A7
:101730002A4629462046FFF76DFE85F31188E9E623
:101740005DB1152284F8702083F3118800212046B2
:10175000D4E91D23FFF75EFEFDE60B2284F870201E
:1017600083F311882B462A4629462046FFF764FE5C
:10177000E3E700BFA43A00089C3A0008A03A00083A
:1017800038B590F870300446002B3ED0063BDAB2F4
:101790000F2A34D80F2B32D8DFE803F03731310865
:1017A000223231313131313131313737856FB0F853
:1017B00086309D4214D2C3681B8AB5FBF3F203FB4B
:1017C00012556DB9202383F311882B462A462946EA
:1017D000FFF732FE85F311880A2384F870300EE09B
:1017E000142384F87030202383F3118800232046CB
:1017F0001A461946FFF70EFE002383F3118838BD01
:10180000C36F03B198470023E7E70021204601F0AA
:101810006BFB0021204601F05BFB63681B6813B182
:101820000621204698470623D7E7000010B590F818
:1018300070300446142B29D017D8062B05D001D8B8
:101840001BB110BD093B022BFBD80021204601F043
:101850004BFB0021204601F03BFB63681B6813B182
:10186000062120469847062319E0152BE9D10B23C2
:1018700080F87030202383F3118800231A4619461C
:10188000FFF7DAFD002383F31188DAE7C3689B6969
:101890005B68002BD5D1C36F03B19847002384F850
:1018A0007030CEE7024B0022C3E900339A607047E4
:1018B000B4230020002382680374054B1B689968D9
:1018C0009142FBD25A6803604260106058607047D2
:1018D000B423002008B5202383F31188037C032B55
:1018E00005D0042B0DD02BB983F3118808BD4369B3
:1018F00000221A604FF0FF334361FFF7DBFF002344
:10190000F2E7D0E9003213605A60F3E700238268FF
:101910000374054B1B6899689142FBD85A680360B1
:101920004260106058607047B4230020054B19696D
:1019300008741868026853601A6018610123037400
:10194000FEF744BDB42300204B1C30B5044687B0DD
:101950000A4D10D02B6901A8094A00F025F920464C
:10196000FFF7E4FF049B13B101A800F059F92B69BC
:10197000586907B030BDFFF7D9FFF8E7B42300205E
:10198000D518000838B50C4D044641612B698168B3
:101990009A68914203D8BDE83840FFF78BBF1846DC
:1019A000FFF7B4FF01232C61014623742046BDE8F4
:1019B0003840FEF70BBD00BFB4230020044B1A686B
:1019C0001B6990689B68984294BF00200120704773
:1019D000B423002010B5084C236820691A685460AD
:1019E0002260012223611A74FFF790FF01462069EB
:1019F000BDE81040FEF7EABCB423002008B5FFF7AD
:101A0000DDFF18B1BDE80840FFF7E4BF08BD0000E6
:101A1000FFF7E0BFFEE7000010B50C4CFFF742FFF8
:101A200000F0B4F880220A49204600F03BF8012378
:101A300044F8180C037400F09BFC002383F3118816
:101A400062B60448BDE8104000F04CB8DC2300202A
:101A5000A83A0008B83A000800F01CB9EFF311806A
:101A600020B9EFF30583202282F31188704700002C
:101A700010B530B9EFF30584C4F3080414B180F352
:101A8000118810BDFFF7BAFF84F31188F9E7000051
:101A9000034A516853685B1A9842FBD8704700BFED
:101AA000001000E082600222028270478368A3F186
:101AB0007C0243F80C2C026943F83C2C426943F841
:101AC000382C074A43F81C2CC268A3F1180043F8CD
:101AD000102C022203F8082C002203F8072C704770
:101AE000E503000810B5202383F31188FFF7DEFF1C
:101AF00000210446FFF746FF002383F311882046A8
:101B000010BD0000024B1B6958610F20FFF70EBF8C
:101B1000B4230020202383F31188FFF7F3BF0000D4
:101B200008B50146202383F311880820FFF70CFF36
:101B3000002383F3118808BD49B1064B42681B6935
:101B400018605A60136043600420FFF7FDBE4FF039
:101B5000FF307047B42300200368984206D01A680B
:101B60000260506018465961FFF7A4BE704700003C
:101B700038B504460D462068844200D138BD03685C
:101B800023605C604561FFF795FEF4E7054B4FF07D
:101B9000FF3103F11402C3E905220022C3E9071251
:101BA000704700BFB423002070B51C4E05460C469C
:101BB000C0E9032301F0B4FB334653F8142F9A42D3
:101BC0000DD130620A2C2CBF00190A302A60C5E9F9
:101BD0000124C6E90555BDE8704001F08BBB316AB0
:101BE000431AE31838BF1C469368A34202D9081968
:101BF00001F090FB73699A6894420CD85A68AC6003
:101C00002B606A6015609A685D60121B9A604FF0E5
:101C1000FF33F36170BDA41A1B68ECE7B423002006
:101C200038B51B4C636998420DD08168D0E9003209
:101C300013605A600022C2609A680A449A604FF0AA
:101C4000FF33E36138BD03682246002142F8143FA8
:101C500093425A60C16003D1BDE8384001F054BBE3
:101C60009A688168256A0A449A6001F059FB6369A1
:101C7000411B9A688A42E5D9AB181D1A206A092DC2
:101C800098BF01F10A02BDE83840104401F042BBA0
:101C9000B42300202DE9F041184C002704F114066C
:101CA000656901F03DFB236AAA68C11A8A4215D80A
:101CB0001344D5F80C802362D5E9003213605A60D2
:101CC0006369EF60B34201D101F01EFB87F3118815
:101CD0002869C047202383F31188E1E76169B14295
:101CE00009D013441B1ABDE8F0410A2B2CBFC018C1
:101CF0000A3001F00FBBBDE8F08100BFB423002023
:101D000000207047FEE70000704700004FF0FF30F2
:101D10007047000002290CD0032904D0012907488C
:101D200018BF00207047032A05D8054800EBC20001
:101D30007047044870470020704700BF9C3B000874
:101D40003C220020503B000870B59AB0054608467A
:101D5000144601A900F0C2F801A8FFF785F8431C5A
:101D60000022C6B25B001046C5E90034237003238D
:101D7000023404F8013C01ABD1B202348E4201D8E6
:101D80001AB070BD13F8011B013204F8010C04F8FD
:101D9000021CF1E708B5202383F311880348FFF7FD
:101DA00067FA002383F3118808BD00BF7025002067
:101DB00090F8803003F01F02012A07D190F88120AB
:101DC0000B2A03D10023C0E91D3315E003F06003A3
:101DD000202B08D1B0F884302BB990F88120212A2B
:101DE00003D81F2A04D8FFF725BA222AEBD0FAE736
:101DF000034A426707228267C3670120704700BF1A
:101E00003322002007B5052917D8DFE801F019169D
:101E100003191920202383F31188104A012101900E
:101E2000FFF7CEFA019802210D4AFFF7C9FA0D48D3
:101E3000FFF7EAF9002383F3118803B05DF804FB90
:101E4000202383F311880748FFF7B4F9F2E7202332
:101E500083F311880348FFF7CBF9EBE7F03A00086A
:101E6000143B00087025002038B50C4D0C4C2A4658
:101E70000C4904F10800FFF767FF05F1CA0204F1FD
:101E800010000949FFF760FF05F5CA7204F1180058
:101E90000649BDE83840FFF757BF00BF483E002065
:101EA0003C220020D03A0008DA3A0008E53A00085F
:101EB00070B5044608460D46FEF7D6FFC6B220466A
:101EC000013403780BB9184670BD32462946FEF737
:101ED000B7FF0028F3D10120F6E700002DE9F84F05
:101EE00005460C46FEF7C0FF2C49C6B22846FFF750
:101EF000DFFF08B10536F6B229492846FFF7D8FFBB
:101F000008B11036F6B2632E0DD8DFF89080DFF8F6
:101F10009090244FDFF894A0DFF894B02E7846B963
:101F20002670BDE8F88F29462046BDE8F84F01F03D
:101F30008BBD252E2ED1072241462846FEF780FF75
:101F400070B9DBF8003007350C3444F80C3CDBF892
:101F5000043044F8083CDBF8083044F8043CDDE782
:101F6000082249462846FEF76BFF98B9A21C0E4B83
:101F7000197802320909C95D02F8041C13F8011B23
:101F800001F00F015345C95D02F8031CF0D118346C
:101F90000835C3E7013504F8016BBFE7BC3B000817
:101FA000E53A0008D13B000800E8F11F0CE8F11FFA
:101FB000C43B0008BFF34F8F044B1A695107FCD193
:101FC000D3F810215207F8D1704700BF002000520B
:101FD00008B50D4B1B78ABB9FFF7ECFF0B4BDA687C
:101FE000D10704D50A4A5A6002F188325A60D3F800
:101FF0000C21D20706D5064AC3F8042102F1883223
:10200000C3F8042108BD00BFA640002000200052F4
:102010002301674508B5114B1B78F3B9104B1A69BA
:10202000510703D5DA6842F04002DA60D3F8102194
:10203000520705D5D3F80C2142F04002C3F80C2119
:10204000FFF7B8FF064BDA6842F00102DA60D3F816
:102050000C2142F00102C3F80C2108BDA64000206B
:10206000002000520F289ABF00F580604004002035
:10207000704700004FF40030704700001020704798
:102080000F2808B50BD8FFF7EDFF00F50033026805
:10209000013204D104308342F9D1012008BD00206F
:1020A000FCE700000F2870B5054645D8FFF7D6FCC1
:1020B000224CFFF77FFF0646FFF78AFF4FF0FF3302
:1020C000072D6361C4F8143120D82361FFF772FF34
:1020D0002B0243F02403E360E36843F08003E360F2
:1020E00023695A07FCD42846FFF764FF4FF40031F8
:1020F000FFF7B8FF00F002F93046FFF78BFFFFF75C
:10210000B7FC2846BDE87040FFF7BABFC4F81031ED
:10211000FFF750FFA5F108031B0243F02403C4F8A6
:102120000C31D4F80C3143F08003C4F80C31D4F8EE
:1021300010315B07FBD4D6E7002070BD00200052B1
:102140002DE9F84F40EA020305460C461746D8062B
:1021500002D00020BDE8F88F27F01F07DFF8D4B0C9
:10216000FFF736FF2744BC4203D10120FFF752FF9F
:10217000F0E720222946204601F056FC10B9203510
:102180002034F0E72B4605F120021E68711CE0D1D7
:1021900004339A42F9D1FFF761FC05F17843234AF1
:1021A000B3F5801F224B28BF9A4603F1040338BFC2
:1021B0009046A2F1080228BF9846A3F108033ABF4F
:1021C0009146DA469946FFF7F5FEC8F80060A5EBA0
:1021D000040CD9F8002004F11C0142F00202C9F8F5
:1021E0000020221FDAF8006016F00506FAD152F836
:1021F000043F8A424CF80230F4D1BFF34F8FFFF70F
:10220000D9FE4FF0FF32C8F80020D9F8002022F0A4
:102210000202C9F80020FFF72BFC202221462846A5
:1022200001F002FC0028AAD030469FE7142000529B
:10223000102100521020005210B5084C237828B10C
:102240001BB9FFF7C5FE0123237010BD002BFCD086
:102250002070BDE81040FFF7DDBE00BFA6400020A3
:102260000244074BD2B210B5904200D110BD441CBD
:1022700000B253F8200041F8040BE0B2F4E700BFCD
:10228000504000580E4B30B51C6F240405D41C6F11
:102290001C671C6F44F400441C670A4C024423680A
:1022A000D2B243F480732360074B904200D130BD1B
:1022B000441C51F8045B00B243F82050E0B2F4E74C
:1022C00000440258004802585040005807B5012207
:1022D00001A90020FFF7C4FF019803B05DF804FBDB
:1022E00013B50446FFF7F2FFA04205D0012201A971
:1022F00000200194FFF7C6FF02B010BD0144BFF3F8
:102300004F8F064B884204D3BFF34F8FBFF36F8FBD
:102310007047C3F85C022030F4E700BF00ED00E036
:1023200000207047034B1A681AB9034AD2F8D02428
:102330001A607047A84000200040025808B5FFF717
:10234000F1FF024B1868C0F3806008BDA840002070
:10235000EFF30983054968334A6B22F001024A63AF
:1023600083F30988002383F31188704700EF00E0AE
:10237000202080F3118862B60D4B0E4AD96821F4F3
:10238000E0610904090C0A430B49DA60D3F8FC2028
:1023900042F08072C3F8FC20084AC2F8B01F1168EE
:1023A00041F0010111601022DA7783F822007047B2
:1023B00000ED00E00003FA0555CEACC5001000E0CA
:1023C000202310B583F311880E4B5B6813F4006370
:1023D00014D0F1EE103AEFF309844FF08073683CAB
:1023E000E361094BDB6B236684F30988FFF7E6FAA8
:1023F00010B1064BA36110BD054BFBE783F31188B9
:10240000F9E700BF00ED00E000EF00E0F70300088F
:10241000FA03000870B5BFF34F8FBFF36F8F1A4AEE
:102420000021C2F85012BFF34F8FBFF36F8F536973
:1024300043F400335361BFF34F8FBFF36F8FC2F884
:102440008410BFF34F8FD2F8803043F6E074C3F3AB
:10245000C900C3F34E335B0103EA0406014646EAB2
:1024600081750139C2F86052F9D2203B13F1200F77
:10247000F2D1BFF34F8F536943F480335361BFF3FD
:102480004F8FBFF36F8F70BD00ED00E0FEE70000DF
:102490000A4B0B480B4A90420BD30B4BC11EDA1C64
:1024A000121A22F003028B4238BF00220021FEF7ED
:1024B000E3BC53F8041B40F8041BECE7B43D0008F0
:1024C0007C4200207C4200207C42002070470000BB
:1024D00070B5D0E9244300224FF0FF359E6804EB2D
:1024E00042135101D3F80009002805DAD3F8000996
:1024F00040F08040C3F80009D3F8000B002805DA4B
:10250000D3F8000B40F08040C3F8000B0132631891
:102510009642C3F80859C3F8085BE0D24FF00113A4
:10252000C4F81C3870BD000000EB8103D3F80CC068
:102530002DE9F043DCF814204E1CD0F89050D2F86E
:1025400000E005EB063605EB4118506870450AD3EC
:102550000122D5F8343802FA01F123EA0101C5F865
:102560003418BDE8F083AEEB0003BCF81040A34282
:1025700028BF2346D8F81849A4B2B3EB840FF0D88B
:102580009468A4F1040959F8047F3760A4EB0907A3
:102590001F44042FF7D81C44034494605360D4E7CD
:1025A000890141F02001016103699B06FCD41220DE
:1025B000FFF76EBA10B50A4C2046FEF7DFFE094B56
:1025C000C4F89030084BC4F89430084C2046FEF70D
:1025D000D5FE074BC4F89030064BC4F8943010BDBC
:1025E000AC40002000000840083C000848410020A2
:1025F00000000440143C000870B503780546012B28
:102600005DD1494BD0F89040984259D1474B0E21AB
:102610006520D3F8D82042F00062C3F8D820D3F860
:10262000002142F00062C3F80021D3F80021D3F862
:10263000802042F00062C3F88020D3F8802022F08E
:102640000062C3F88020D3F8803000F071FC384B72
:10265000E360384BC4F800380023D5F89060C4F824
:10266000003EC02323604FF40413A3633369002B9F
:10267000FCDA01230C203361FFF70AFA3369DB0728
:10268000FCD41220FFF704FA3369002BFCDA002691
:102690002846A660FFF71CFF6B68C4F81068DB686B
:1026A000C4F81468C4F81C68002B3AD1224BA3610B
:1026B0004FF0FF336361A36843F00103A36070BD73
:1026C0001E4B9842C8D1194B0E214D20D3F8D8206B
:1026D00042F00072C3F8D820D3F8002142F0007213
:1026E000C3F80021D3F80021D3F8802042F0007213
:1026F000C3F88020D3F8802022F00072C3F8802035
:10270000D3F88020D3F8D82022F08062C3F8D820F4
:10271000D3F8002122F08062C3F80021D3F8003101
:1027200093E7074BC3E700BFAC40002000440258CA
:102730004014004003002002003C30C0484100200B
:10274000083C30C0F8B5D0F89040054600214FF065
:1027500000662046FFF724FFD5F8941000234FF0C1
:1027600001128F684FF0FF30C4F83438C4F81C28C9
:1027700004EB431201339F42C2F80069C2F8006BB8
:10278000C2F80809C2F8080BF2D20B68D5F89020FD
:10279000C5F89830636210231361166916F01006AD
:1027A000FBD11220FFF774F9D4F8003823F4FE634C
:1027B000C4F80038A36943F4402343F01003A36135
:1027C0000923C4F81038C4F814380B4BEB604FF0F1
:1027D000C043C4F8103B094BC4F8003BC4F810696F
:1027E000C4F80039D5F8983003F1100243F480138F
:1027F000C5F89820A362F8BDE43B000840800010B3
:10280000D0F8902090F88A10D2F8003823F4FE63B4
:1028100043EA0113C2F80038704700002DE9F8437D
:1028200000EB8103D0F890500C468046DA680FFA2E
:1028300081F94801166806F00306731E022B05EBAA
:1028400041134FF0000194BFB604384EC3F8101B7B
:102850004FF0010104F1100398BF06F1805601FA10
:1028600003F3916998BF06F5004600293AD0578ACC
:1028700004F15801374349016F50D5F81C180B4338
:102880000021C5F81C382B180127C3F81019A740E0
:102890005369611E9BB3138A928B9B08012A88BFE0
:1028A0005343D8F89820981842EA034301F14002B4
:1028B0002146C8F89800284605EB82025360FFF7CE
:1028C0006FFE08EB8900C3681B8A43EA84534834CF
:1028D0001E4364012E51D5F81C381F43C5F81C78DF
:1028E000BDE8F88305EB4917D7F8001B21F4004138
:1028F000C7F8001BD5F81C1821EA0303C0E704F150
:102900003F030B4A2846214605EB83035A60FFF735
:1029100047FE05EB4910D0F8003923F40043C0F816
:102920000039D5F81C3823EA0707D7E700800010E4
:1029300000040002D0F894201268C0F89820FFF735
:10294000C7BD00005831D0F8903049015B5813F4EE
:10295000004004D013F4001F0CBF02200120704778
:102960004831D0F8903049015B5813F4004004D04E
:1029700013F4001F0CBF02200120704700EB8101FF
:10298000CB68196A0B6813604B685360704700008E
:1029900000EB810330B5DD68AA691368D36019B90B
:1029A000402B84BF402313606B8A1468D0F89020BA
:1029B0001C4402EB4110013C09B2B4FBF3F4634345
:1029C000033323F0030343EAC44343F0C043C0F896
:1029D000103B2B6803F00303012B0ED1D2F808380B
:1029E00002EB411013F4807FD0F8003B14BF43F09A
:1029F000805343F00053C0F8003B02EB4112D2F881
:102A0000003B43F00443C2F8003B30BD2DE9F041E8
:102A1000D0F8906005460C4606EB4113D3F8087BCE
:102A20003A07C3F8087B08D5D6F814381B0704D535
:102A300000EB8103DB685B689847FA071FD5D6F87F
:102A40001438DB071BD505EB8403D968CCB98B6937
:102A5000488A5A68B2FBF0F600FB16228AB9186859
:102A6000DA6890420DD2121AC3E90024202383F3BE
:102A7000118821462846FFF78BFF84F31188BDE8B3
:102A8000F081012303FA04F26B8923EA02036B81CC
:102A9000CB68002BF3D021462846BDE8F04118470B
:102AA00000EB81034A0170B5DD68D0F890306C69A5
:102AB0002668E66056BB1A444FF40020C2F810099D
:102AC0002A6802F00302012A0AB20ED1D3F80808DC
:102AD00003EB421410F4807FD4F8000914BF40F0D7
:102AE000805040F00050C4F8000903EB4212D2F8C5
:102AF000000940F00440C2F800090122D3F834086C
:102B000002FA01F10143C3F8341870BD19B9402E1F
:102B100084BF4020206020681A442E8A8419013C1A
:102B2000B4FBF6F440EAC44040F00050C6E70000B1
:102B30002DE9F041D0F8906004460D4606EB4113B4
:102B4000D3F80879C3F80879FB071CD5D6F81038F4
:102B5000DA0718D500EB8103D3F80CC0DCF8143089
:102B6000D3F800E0DA6896451BD2A2EB0E024FF0D4
:102B700000081A60C3F80480202383F31188FFF74C
:102B80008FFF88F311883B0618D50123D6F8342827
:102B9000AB40134212D029462046BDE8F041FFF772
:102BA000C3BC012303FA01F2038923EA0203038170
:102BB000DCF80830002BE6D09847E4E7BDE8F08168
:102BC0002DE9F84FD0F8905004466E69AB691E406D
:102BD00016F480586E6103D0BDE8F84FFEF73EBC96
:102BE000002E12DAD5F8003E9F0705D0D5F8003E3A
:102BF00023F00303C5F8003ED5F80438204623F03F
:102C00000103C5F80438FEF755FC300505D520460C
:102C1000FFF75EFC2046FEF73DFCB1040CD5D5F86D
:102C2000083813F0060FEB6823F470530CBF43F41D
:102C3000105343F4A053EB60320704D56368DB689C
:102C40000BB120469847F30200F1BA80B70226D5AF
:102C5000D4F8909000274FF0010A09EB4712D2F800
:102C6000003B03F44023B3F5802F11D1D2F8003B91
:102C7000002B0DDA62890AFA07F322EA0303638163
:102C800004EB8703DB68DB6813B1394620469847BD
:102C90000137D4F89430FFB29B689F42DDD9F0062B
:102CA00019D5D4F89000026AC2F30A1702F00F0394
:102CB00002F4F012B2F5802F00F0CC80B2F5402F74
:102CC00009D104EB8303002200F58050DB681B6A06
:102CD000974240F0B2803003D5F8185835D5E90353
:102CE00003D500212046FFF791FEAA0303D5012159
:102CF0002046FFF78BFE6B0303D502212046FFF72A
:102D000085FE2F0303D503212046FFF77FFEE8024F
:102D100003D504212046FFF779FEA90203D505213A
:102D20002046FFF773FE6A0203D506212046FFF70F
:102D30006DFE2B0203D507212046FFF767FEEF014A
:102D400003D508212046FFF761FE700340F1A980FA
:102D5000E90703D500212046FFF7EAFEAA0703D5BD
:102D600001212046FFF7E4FE6B0703D50221204630
:102D7000FFF7DEFE2F0703D503212046FFF7D8FE1D
:102D8000EE0603D504212046FFF7D2FEA80603D5A0
:102D900005212046FFF7CCFE690603D50621204613
:102DA000FFF7C6FE2A0603D507212046FFF7C0FE1F
:102DB000EB0576D520460821BDE8F84FFFF7B8BEF1
:102DC000D4F8909000274FF0010AD4F894305FFABD
:102DD00087FB9B689B453FF639AF09EB4B13D3F854
:102DE000002902F44022B2F5802F24D1D3F8002923
:102DF000002A20DAD3F8002942F09042C3F80029D3
:102E0000D3F80029002AFBDB5946D4F89000FFF7DD
:102E1000C7FB22890AFA0BF322EA0303238104EB9E
:102E20008B03DB689B6813B1594620469847594687
:102E30002046FFF779FB0137C7E7910701D1D0F8AA
:102E40000080072A02F101029CBF03F8018B4FEAC0
:102E500018283DE704EB830300F58050DA68D2F8C8
:102E600018C0DCF80820DCE9001CA1EB0C0C0021E8
:102E70008F4208D1DB689B699A683A449A605A6825
:102E80003A445A6027E711F0030F01D1D0F80080CF
:102E90008C4501F1010184BF02F8018B4FEA18282B
:102EA000E6E7BDE8F88F000008B50348FFF788FEA5
:102EB000BDE80840FFF784BAAC40002008B50348DD
:102EC000FFF77EFEBDE80840FFF77ABA48410020D0
:102ED000D0F8903003EB4111D1F8003B43F40013DC
:102EE000C1F8003B70470000D0F8903003EB41116F
:102EF000D1F8003943F40013C1F8003970470000DD
:102F0000D0F8903003EB4111D1F8003B23F40013CB
:102F1000C1F8003B70470000D0F8903003EB41113E
:102F2000D1F8003923F40013C1F8003970470000CC
:102F3000090100F16043012203F56143C9B283F83E
:102F4000001300F01F039A4043099B0003F1604304
:102F500003F56143C3F880211A60704730B504332C
:102F6000039C0172002104FB0325C160C0E90653E4
:102F7000049B0363059BC0E90000C0E90422C0E98B
:102F80000842C0E90A11436330BD00000022416AD3
:102F9000C260C0E90411C0E90A226FF00101FEF726
:102FA000E7BD0000D0E90432934201D1C2680AB9FA
:102FB000181D704700207047036919600021C2681E
:102FC0000132C260C269134482699342036124BF23
:102FD000436A0361FEF7C0BD38B504460D46E36899
:102FE0003BB162690020131D1268A3621344E362BF
:102FF00007E0237A33B929462046FEF79DFD0028D5
:10300000EDDA38BD6FF00100FBE70000C368C2696C
:10301000013BC3604369134482699342436124BF07
:10302000436A436100238362036B03B1184770470F
:1030300070B52023044683F31188866A3EB9FFF7F2
:10304000CBFF054618B186F31188284670BDA36AE8
:10305000E26A13F8015B9342A36202D32046FFF7B2
:10306000D5FF002383F31188EFE700002DE9F84F27
:1030700004460E46174698464FF0200989F31188FA
:103080000025AA46D4F828B0BBF1000F09D141466B
:103090002046FFF7A1FF20B18BF311882846BDE839
:1030A000F88FD4E90A12A7EB050B521A934528BFF3
:1030B0009346BBF1400F1BD9334601F1400251F852
:1030C000040B914243F8040BF9D1A36A4036403512
:1030D0004033A362D4E90A239A4202D32046FFF781
:1030E00095FF8AF31188BD42D8D289F31188C9E7C8
:1030F00030465A46FDF79AFEA36A5E445D445B443F
:10310000A362E7E710B5029C0433017204FB0321BC
:10311000C460C0E906130023C0E90A33039B0363BC
:10312000049BC0E90000C0E90422C0E908424363EF
:1031300010BD0000026A6FF00101C260426AC0E97E
:1031400004220022C0E90A22FEF712BDD0E90423BE
:103150009A4201D1C26822B9184650F8043B0B606C
:103160007047002070470000C3680021C269013326
:10317000C3604369134482699342436124BF436A35
:103180004361FEF7E9BC000038B504460D46E3682C
:103190003BB1236900201A1DA262E2691344E36275
:1031A00007E0237A33B929462046FEF7C5FC0028FC
:1031B000EDDA38BD6FF00100FBE70000036919602C
:1031C000C268013AC260C2691344826993420361D2
:1031D00024BF436A036100238362036B03B1184772
:1031E0007047000070B520230D460446114683F356
:1031F0001188866A2EB9FFF7C7FF10B186F31188D0
:1032000070BDA36A1D70A36AE26A01339342A36290
:1032100004D3E16920460439FFF7D0FF002080F392
:103220001188EDE72DE9F84F04460D469046994682
:103230004FF0200A8AF311880026B346A76A4FB9D7
:1032400049462046FFF7A0FF20B187F3118830469A
:10325000BDE8F88FD4E90A073A1AA8EB06079742A7
:1032600028BF1746402F1BD905F1400355F8042B02
:103270009D4240F8042BF9D1A36A40364033A36243
:10328000D4E90A239A4204D3E16920460439FFF7BE
:1032900095FF8BF311884645D9D28AF31188CDE783
:1032A00029463A46FDF7C2FDA36A3D443E443B44ED
:1032B000A362E5E7D0E904239A4217D1C3689BB122
:1032C000836A8BB1043B9B1A0ED01360C368013B29
:1032D000C360C3691A4483699A42026124BF436A86
:1032E0000361002383620123184670470023FBE734
:1032F00000F0DAB8034B002258631A610222DA6048
:10330000704700BF000C0040014B0022DA6070479C
:10331000000C0040014B5863704700BF000C004098
:10332000014B586A704700BF000C00404B68436077
:103330008B688360CB68C3600B6943614B69036230
:103340008B6943620B6803607047000008B53C4B13
:1033500040F2FF713B48D3F888200A43C3F8882025
:10336000D3F8882022F4FF6222F00702C3F88820F5
:10337000D3F88820D3F8E0200A43C3F8E020D3F83C
:1033800008210A43C3F808212F4AD3F8083111460F
:10339000FFF7CCFF00F5806002F11C01FFF7C6FFCC
:1033A00000F5806002F13801FFF7C0FF00F5806092
:1033B00002F15401FFF7BAFF00F5806002F17001DD
:1033C000FFF7B4FF00F5806002F18C01FFF7AEFF5C
:1033D00000F5806002F1A801FFF7A8FF00F580600A
:1033E00002F1C401FFF7A2FF00F5806002F1E001E5
:1033F000FFF79CFF00F5806002F1FC01FFF796FFEC
:1034000002F58C7100F58060FFF790FF00F000F985
:103410000E4BD3F8902242F00102C3F89022D3F869
:10342000942242F00102C3F894220522C3F89820A6
:103430004FF06052C3F89C20054AC3F8A02008BD95
:103440000044025800000258203C000800ED00E053
:103450001F00080308B500F0C9FAFEF7DDFA0F4BAC
:10346000D3F8DC2042F04002C3F8DC20D3F804217A
:1034700022F04002C3F80421D3F80431084B1A6843
:1034800042F008021A601A6842F004021A60FEF75D
:1034900049FFBDE80840FEF7E7BC00BF0044025802
:1034A0000018024870470000114BD3F8E82042F0A2
:1034B0000802C3F8E820D3F8102142F00802C3F84C
:1034C00010210C4AD3F81031D36B43F00803D363B7
:1034D000C722094B9A624FF0FF32DA6200229A61EA
:1034E0005A63DA605A6001225A611A60704700BF5D
:1034F000004402580010005C000C0040094A08B566
:103500001169D3680B40D9B29B076FEA01011161C1
:1035100007D5202383F31188FEF79EFA002383F357
:10352000118808BD000C0040384B4FF0FF31D3F834
:103530008020C3F88010D3F880200022C3F88020B8
:10354000D3F88000D3F88400C3F88410D3F8840043
:10355000C3F88420D3F88400D86F40F0FF4040F4D3
:10356000FF0040F43F5040F03F00D867D86F20F094
:10357000FF4020F4FF0020F43F5020F03F00D867C8
:10358000D86FD3F888006FEA40506FEA5050C3F804
:103590008800D3F88800C0F30A00C3F88800D3F885
:1035A0008800D3F89000C3F89010D3F89000C3F8C7
:1035B0009020D3F89000D3F89400C3F89410D3F877
:1035C0009400C3F89420D3F89400D3F89800C3F87B
:1035D0009810D3F89800C3F89820D3F89800D3F83F
:1035E0008C00C3F88C10D3F88C00C3F88C20D3F86F
:1035F0008C00D3F89C00C3F89C10D3F89C10C3F83F
:103600009C20D3F89C3000F0C9B900BF0044025898
:10361000614B0122C3F80821604BD3F8F42042F03B
:103620000202C3F8F420D3F81C2142F00202C3F8CE
:103630001C210222D3F81C31594BDA605A689104DC
:10364000FCD5584A1A6001229A60574ADA60002273
:103650001A614FF440429A61514B9A699204FCD529
:103660001A6842F480721A604C4B1A6F12F4407F51
:1036700004D04FF480321A6700221A671A6842F0A9
:1036800001021A60454B1A685007FCD500221A61E6
:103690001A6912F03802FBD1012119604FF0804104
:1036A00059605A67414ADA62414A1A611A6842F41B
:1036B00080321A60394B1A689103FCD51A6842F4BB
:1036C00080521A601A689204FCD53A4A3A499A62C2
:1036D00000225A6319633949DA6399635A64384A94
:1036E0001A64384ADA621A6842F0A8521A602B4B00
:1036F0001A6802F02852B2F1285FF9D148229A6183
:103700004FF48862DA6140221A622F4ADA644FF07D
:1037100080521A652D4A5A652D4A9A6532232D4AE0
:103720001360136803F00F03022BFAD11B4B1A69C5
:1037300042F003021A611A6902F03802182AFAD11B
:10374000D3F8DC2042F00052C3F8DC20D3F8042187
:1037500042F00052C3F80421D3F80421D3F8DC204E
:1037600042F08042C3F8DC20D3F8042142F08042CA
:10377000C3F80421D3F80421D3F8DC2042F000423E
:10378000C3F8DC20D3F8042142F00042C3F804213E
:10379000D3F80431704700BF008000510044025844
:1037A0000048025800C000F0020000010000FF01C4
:1037B0000088900812102000630209012C02040006
:1037C00047040508FD0BFF01200000200010E00069
:1037D00000010100002000524FF0B04208B5D2F8BD
:1037E000883003F00103C2F8883023B1044A13681B
:1037F0000BB150689847BDE80840FEF7E1BD00BF37
:10380000FC4100204FF0B04208B5D2F8883003F0F8
:103810000203C2F8883023B1044A93680BB1D06820
:103820009847BDE80840FEF7CBBD00BFFC41002033
:103830004FF0B04208B5D2F8883003F00403C2F864
:10384000883023B1044A13690BB150699847BDE829
:103850000840FEF7B5BD00BFFC4100204FF0B0426C
:1038600008B5D2F8883003F00803C2F8883023B1D5
:10387000044A93690BB1D0699847BDE80840FEF748
:103880009FBD00BFFC4100204FF0B04208B5D2F808
:10389000883003F01003C2F8883023B1044A136A59
:1038A0000BB1506A9847BDE80840FEF789BD00BFDC
:1038B000FC4100204FF0B04310B5D3F8884004F429
:1038C0007872C3F88820A30604D5124A936A0BB114
:1038D000D06A9847600604D50E4A136B0BB1506B43
:1038E0009847210604D50B4A936B0BB1D06B9847D0
:1038F000E20504D5074A136C0BB1506C9847A30539
:1039000004D5044A936C0BB1D06C9847BDE81040C5
:10391000FEF756BDFC4100204FF0B04310B5D3F880
:10392000884004F47C42C3F88820620504D5164A16
:10393000136D0BB1506D9847230504D5124A936D52
:103940000BB1D06D9847E00404D50F4A136E0BB14C
:10395000506E9847A10404D50B4A936E0BB1D06EFC
:103960009847620404D5084A136F0BB1506F98470B
:10397000230404D5044A936F0BB1D06F9847BDE878
:103980001040FEF71DBD00BFFC41002008B5FFF749
:10399000B5FDBDE80840FEF713BD0000062108B5DF
:1039A0000846FFF7C5FA06210720FFF7C1FA0621EE
:1039B0000820FFF7BDFA06210920FFF7B9FA062112
:1039C0000A20FFF7B5FA06211720FFF7B1FA062102
:1039D0002820FFF7ADFA09217A20FFF7A9FA07217D
:1039E0003220BDE80840FFF7A3BA000008B5FFF792
:1039F0009BFD00F00BF8FDF7BFFCFDF791FBFFF717
:103A000051FDBDE80840FFF773BC00000023054AE4
:103A100019460133102BC2E9001102F10802F8D156
:103A2000704700BFFC41002010B5013902449042AC
:103A300001D1002005E0037811F8014FA34201D025
:103A4000181B10BD0130F2E7034611F8012B03F8F3
:103A5000012B002AF9D1704753544D333248373F78
:103A60003F3F0053544D3332483734332F373533CB
:103A700000000000000000009D10000889100008F0
:103A8000C5100008B1100008BD100008A9100008FA
:103A90009510000881100008D110000800000000F7
:103AA00001000000000000006D61696E0000000070
:103AB00069646C6500000000B03A0008F82300203B
:103AC0007025002001000000151A00080000000009
:103AD0004172647550696C6F740025424F415244C5
:103AE000252D424C002553455249414C25000000EC
:103AF0000200000000000000BD1200082D130008A5
:103B000040004000183E0020283E00200200000037
:103B10000000000003000000000000007513000812
:103B20000000000010000000383E002000000000EF
:103B30000100000000000000AC4000200101020074
:103B4000051E0008151D0008B11D0008951D000880
:103B500043000000583B000809024300020100C076
:103B600032090400000102020100052400100105D1
:103B70002401000104240202052406000107058235
:103B8000030800FF09040100020A00000007050104
:103B90000240000007058102400000001200000002
:103BA000A43B000812011001020000400912415715
:103BB00000020102030100000403090425424F41F1
:103BC00052442500466F7865657248373433763144
:103BD0000030313233343536373839414243444589
:103BE0004600000000000000C9140008811700080A
:103BF0002D18000840004000E4410020E44100206E
:103C000001000000F441002080000000400100009D
:103C1000080000000001000000040000080000008F
:103C20000001816A00000000AAAAAAAA000100649B
:103C3000FFFE00000000000000A00A0000000001DC
:103C400000000000AAAAAAAA00000001FFFF0000CD
:103C50000000000000000000000000000000000064
:103C6000AAAAAAAA00000000FFFF000000000000AE
:103C7000000000000000000000000000AAAAAAAA9C
:103C800000000000FFFF0000000000000000000036
:103C90000000000000000000AAAAAAAA000000007C
:103CA000FFFF000000000000000000000000000016
:103CB00000000000AAAAAAAA00000000FFFF00005E
:103CC00000000000000000000000000000000000F4
:103CD000AAAAAAAA00000000FFFF0000000000003E
:103CE000000000000000000000000000AAAAAAAA2C
:103CF00000000000FFFF00000000000000000000C6
:103D00000000000000000000AAAAAAAA000000000B
:103D1000FFFF0000000000000000000000000000A5
:103D200000000000AAAAAAAA00000000FFFF0000ED
:103D30000000000000000000000000000000000083
:103D4000AAAAAAAA00000000FFFF000000000000CD
:103D5000000000000000000041040000000000001E
:103D600000001A0000000000FF000000000000003A
:103D7000583A00083F00000050040000633A000871
:103D80003F000000009600000000080096000000C0
:103D90000008000004000000B83B0008000000001C
:103DA0000000000000000000000000000000000013
:043DB000000000000F
:00000001FF
